:020000020000FC
:0200000027C017
:1000140000C07F937FB7949A959A606494980FBFB9
:100024007F9118957F93C49A6062959A88247EE1A3
:10003400972E7F910895C4986F7D959843987AE0A0
:100044007A9511F0AAD0FCCF439A08950FED0DBF15
:100054007AE07A9511F0A1D0FCCF7CE078BB70EF08
:1000640077BB9BD000E0502E0AEF602E01E8702E83
:100074005AEA56D099D000E002BB0FEF01BB6627C5
:10008400E0E0F3E0CFDF08E008B97894439A0FEF9B
:1000940051D065FD959A65FDC49A66FF03C0C2DF21
:1000A40095986F7BEA9549F4FA9539F4E0E0F3E02A
:1000B40067FF03C05AEA29D06F778A9419F49A9497
:1000C40009F4B9DF06B30C7019D016B31C7001170C
:1000D40001F701D0DECF043019F0083041F0089563
:1000E400042D0F3F11F04394A3D09CDF1FC0042DB7
:1000F400073311F04A949CD095DF18C028EC30E007
:100104003A95F1F72A95D9F70895F894E199FDCF36
:100114005EBB4DBAE29AE19A04E60CD07894089555
:10012400E199FECF5EBBE09A4DB20895E0E0F3E0C2
:10013400606802E39598969A1CD096981AD00A950E
:10014400C9F742BB47FF02C0889A01C08898959AB4
:1001540006B30C70003041F0D1DF16B31C700117E8
:10016400B9F70C30A9F708955DDF0FEA402E60D08F
:10017400DDCF21E036E93A95F1F72A95D9F70895CC
:10018400C698770F08F4C69AC59A0000C59800006F
:100194000895C79A0000C7980895222433243A94F6
:1001A400F1F72A94D9F7089570ECEADFE9DF75ECEA
:1001B400E7DFE6DFE5DFE4DFE3DFE2DFE1DFE0DF27
:1001C40070E0DEDFDDDFDCDFDBDFDADFD9DFD8DFC5
:1001D400D7DFDFDF70EFD4DFD3DF70ECD1DFD0DF28
:1001E400CFDFCEDFCDDFCCDFCBDFCADF72E0C8DF0D
:1001F400C7DFC6DFC5DFC4DFC3DFC2DFC1DFC9DFDE
:1002040017D070E0BDDFBCDF70E0BADFB9DFB8DF64
:10021400B7DFB6DFB5DFB4DFB3DF73E0B1DFB0DF84
:10022400AFDFAEDFADDFACDFABDFAADFB2DF089557
:10023400B0E0A42DD3E0C9E38894CA1FDB1F0D2FBF
:10024400DD0FDD0FDD0FDD0FD07C752D7F737D2B72
:10025400572E000F000F000F000F000F000F007C3F
:100264006624602A0C2F069506950F73602ACC0F1E
:10027400CC0FCC0FCC0FCC0FCC0FC07C072D0F7341
:100284000C2B702E752D7CDF7BDF762D79DF78DFEC
:1002940077DF76DF75DF74DF73DF72DF772D70DF72
:1002A4006FDF6EDF6DDF6CDF6BDF6ADF69DF71DFED
:0202B4000895AB
:00000001FF
